:020000040000FA
:10000000CCB0B3D4C9DF0000000000000000000045
:1000100000000000030000000002000014000000C7
:100020000160704747F6954CC0F60E0C604748F6E5
:10003000652CC0F60D0C60474AF2C31CC0F60D0CCF
:10004000604748F6293CC0F60D0C604748F6793CFD
:10005000C0F60D0C604749F2EB5CC0F60D0C604732
:1000600049F2052CC0F60D0C604748F65F7CC0F6DF
:100070000D0C604748F6E97CC0F60D0C60474CF269
:10008000BD0CC0F60E0C604748F6F94CC0F60D0CDE
:10009000604748F2CD2CC0F60D0C604748F29F3CFB
:1000A000C0F60D0C604748F6F72CC0F60D0C604703
:1000B00047F6897CC0F60D0C60474CF27B0CC0F60D
:1000C0000D0C60474CF2151CC0F60D0C60474BF64A
:1000D0002F6CC0F60D0C604744F6E55CC0F6020CD0
:1000E00060474DF6492CC0F60D0C604744F65F5C46
:1000F000C0F6020C60474BF6CF5CC0F60D0C6047B3
:100100004BF6B15CC0F60D0C60474BF64F4CC0F699
:100110000D0C60474BF6F90CC0F60D0C60474BF226
:10012000610CC0F60D0C604744F6851CC0F6020C4D
:1001300060474FF6F12CC0F60D0C604740F2812C61
:10014000C0F6020C604740F2852CC0F6020C6047F6
:1001500048F6FF0CC0F60D0C604748F6D50CC0F60B
:100160000D0C604748F2F15CC0F60D0C604745F29B
:10017000C14CC0F6020C60472DE9F04D8CB08046B2
:1001800000200B900A90D8F808000990D8F80C00CD
:100190000890D8F834B0D8F838000790142102A895
:1001A000FFF740FF4046FFF742FF1820FFF744FFEC
:1001B00001905846FFF745FF0798FFF747FFD8F82B
:1001C000C00100287ED01E2619270798FFF739FFA7
:1001D000791E701ECA231A46FFF73DFF5846FFF7E7
:1001E00030FF791E701ECA231A46FFF739FF4FF001
:1001F000000A002468E0002561E004EBC40101EB83
:10020000041105EB410101EB4101D8F8C00100EBFD
:10021000010A9AF80000012808D107EB840106EBD7
:10022000850004231A46FFF71BFF47E09AF80000F9
:1002300002280AD107EB8402511C06EB8502501CF0
:1002400002231A46FFF70CFF38E09AF80000032853
:1002500008D107EB840106EB850004231A46FFF75B
:10026000FAFE2BE09AF80000042827D106EB85035C
:10027000DA1C07EB8403591C06EB8500FFF7F5FE3B
:1002800006EB8503DA1C07EB8403991C06EB85005B
:10029000FFF7EBFE07EB8403DA1C07EB840106EBA8
:1002A0008503581CFFF7E6FE07EB8403DA1C07EB17
:1002B000840106EB8503981CFFF7DCFE6D1C322DD4
:1002C0009BDB00E01CE0641C322C94DBD8F8C001FE
:1002D00000F580500DA1D0F8502D02A8FFF7CFFEF9
:1002E0001E224FF48A7102A8FFF7CEFED8F8C4018F
:1002F00028B13C224FF48A7107A0FFF7C5FE00BF6A
:100300000198FFF799FE0CB0BDE8F08DB7D6CAFD95
:10031000A3BA256400000000D4DDCDA3D6D0000030
:1003200070B5044600F0CAF90546D4F8C00100F0E3
:100330005AFA2046FFF7ADFE002004494944086000
:1003400000F0EAF9284600F0E1F970BD080000006D
:100350002DE9FC41044600255CB1D4E902010023EB
:100360001A46CDE900011946204600F03FF905463E
:100370000EE0FFF793FEC668FFF790FE8768002344
:100380001A4619461846CDE9007600F02FF90546C1
:1003900004F13C012846FFF786FE2846FFF788FE59
:1003A0002846BDE8FC8100002DE9FC4704460D46C7
:1003B00000F084F906464FF00008002728680A2854
:1003C0007ED2DFE800F0EB050999EBAFEB9CEB4E3A
:1003D0002046FFF7D1FEE6E01E2000906E234FF48A
:1003E000AF72002101902046FFF767FEC4F8C801F4
:1003F00070A1D4F8C801FFF765FE1E200090C82345
:100400004FF4AF72002101902046FFF756FEC4F86A
:10041000CC0169A1D4F8CC01FFF754FE1E20009056
:10042000A0234FF49672002101902046FFF745FE6D
:10043000C4F8D00161A1D4F8D001FFF743FE1E201B
:100440000090A0234FF4C872002101902046FFF7CE
:1004500034FEC4F8D4015AA1D4F8D401FFF732FE17
:10046000A1E0E868D4F8BC11884244D1D4F8C401B2
:10047000002840D1D4F8C00100F043FB40BBD4F8C1
:10048000BC01FFF724FE8020FFF726FE8246D4F849
:10049000C00100F580504BA1D0F8502D5046FFF719
:1004A000EEFD4EA352464FA12046FFF71AFE5046DE
:1004B000FFF71CFED4F8C00100F0F0FA204600E07F
:1004C0006CE0D4F8D811FFF716FEC4F8BC0100BFE9
:1004D000D4F8D801B0F5967F0ADDD4F8D801401ED3
:1004E000C4F8D801D4F8D811D4F8BC01FFF708FE3D
:1004F0002046FFF70AFE56E0D5F80C8053E0EF687F
:10050000B86805280BD1D4F8C40108B9012000E06F
:100510000020C4F8C4012046FFF7F7FD00E000BF4B
:1005200000BF40E0E868012802D0022833D100E093
:1005300032E0286901282DD16868D4F8C8118842B2
:1005400005D10321D4F8C00100F0E5FA1FE0686886
:10055000D4F8CC11884205D10421D4F8C00100F0B0
:10056000DAFA14E06868D4F8D011884205D1022183
:10057000D4F8C00100F0CFFA09E06868D4F8D411CB
:10058000884204D10121D4F8C00100F0C4FA204609
:10059000FFF7C0FD00E000BF00BF04E02946204691
:1005A000FFF7BDFD00BF00BF304600F0AFF8BDE86B
:1005B000FC870000C9CF0000CFC20000D7F30000C5
:1005C000D3D20000D3CECFB7BDE1CAF80AB5B1C7C8
:1005D000B0B7D6CAFDA3BA2564000000C8B7B6A854
:1005E00000000000CCE1CABE000000002DE9FE4F73
:1005F00006460D4617469846DDE90CAB0DB91D4D74
:100600007D444FF4EE70FFF767FD044664B34FF48A
:10061000EE7200212046FFF787FD3B462A46314611
:1006200020468DE8000DFFF784FD20B92046FFF736
:100630005DFD002418E010A0606101206066124892
:100640007844C4F8D0004FF42F70C4F8D801204685
:10065000D4F8D811FFF74FFDC4F8BC0100F0B8F88A
:10066000C4F8C00100F06EF8084848440460204611
:10067000BDE8FE8FA5FDFFFF57494E5F536E616BCE
:100680006553747275637400DDFCFFFF08000000A1
:1006900070B5054600F012F8044607484844006863
:1006A00020B1054848440068FFF73AFE204600F0B4
:1006B0002DF8002070BD00000800000010B5FFF705
:1006C0003DFD0446034878440068FFF73CFD2046A2
:1006D00010BD00006A04000070B50446FFF72EFD4F
:1006E0000546294606487844FFF79AFC05484844E1
:1006F000046005487844034949440968486170BD6D
:100700004A0400000400000099FFFFFF10B50446F2
:100710002046FFF718FD10BD09484844006868B13D
:10072000074848440068806940B10548484400686B
:100730008069401E02494944096888617047000089
:100740000400000006484844006840B1044848449A
:1007500000688069401C0249494409688861704703
:100760000400000070B505462846FFF7B5FFFFF707
:10077000E9FF002411A10020FFF7EAFC04460CB9B0
:10078000012000E0002068B10FA10020FFF7E0FC8D
:1007900006463046FFF7DCFD044608A12046FFF779
:1007A000DCFC06E02146A06FFFF7DCFC2046FFF7EB
:1007B0007FFCFFF7B1FF002070BD000077696E5F1E
:1007C000736E616B65000000686F6D65000000006E
:1007D00010B541F65C50FFF77FFC0446204600F060
:1007E0005DF9204610BD10B5044614B12046FFF750
:1007F0007DFC10BD70B5014641F65A50425C401C6C
:10080000435C03EBC30000EB031002EB400000EB82
:100810004000451800202870FF206870A870002450
:10082000312B19DA581C00EBC00606EB001002EB66
:10083000400000EB40004418607890420CD1A07852
:10084000984209D141F65A504254581CC6B241F65A
:100850005B504654012070BD002B19DD581E00EB83
:10086000C00606EB001002EB400000EB400044180D
:10087000607890420CD1A078984209D141F65A5044
:100880004254581EC6B241F65B5046540120E2E77E
:10089000002A18DD501E03EBC30606EB031600EB1F
:1008A000460000EB40004418607890420BD1A078DD
:1008B000984208D1501EC6B241F65A504654401CC8
:1008C00043540120C7E7312A18DA03EBC30000EBD9
:1008D0000316501C00EB460000EB40004418607803
:1008E00090420BD1A078984208D1501CC6B241F674
:1008F0005A504654401C43540120ACE70020AAE75C
:100900002DE9F041044641F650500159001F0059AD
:1009100040F6C412101A0A38814202DD0020BDE8F8
:10092000F08100BFFFF723FC3221B0FBF1F201FBA5
:100930001206FFF71CFC3221B0FBF1F201FB12079B
:1009400007EBC70000EB071006EB400000EB400090
:100950000519287818B9042028700120DFE7E1E79D
:100960002DE9F04D044641F65850065D401C075DE8
:1009700007EBC70000EB071006EB400000EB400060
:1009800000EB040B03208BF800002046FFF732FF3A
:1009900010B90020BDE8F08DB046BA4641F654507B
:1009A0000059012802D1701CC6B216E041F654501D
:1009B0000059022802D1701EC6B20EE041F6545012
:1009C0000059032802D1781EC7B206E041F6545000
:1009D0000059042801D1781CC7B2322E01DA322F17
:1009E00001DB0020D6E707EBC70000EB071006EBA2
:1009F000400000EB400005192878C0B12878042891
:100A000013D141F650500059401C41F65051085145
:100A10000220287085F8018085F802A0204600F0A9
:100A200013F82046FFF76CFF07E00020B2E7022032
:100A3000287085F8018085F802A041F658500655C7
:100A4000401C07550120A5E710B5014641F65A5054
:100A5000425C401C435C03EBC30000EB031002EB61
:100A6000400000EB400044186278A378322A01DA93
:100A7000322B01DB002010BD03EBC30000EB0310A1
:100A800002EB400000EB400044180320207041F6C8
:100A90005A504254401C43540120ECE770B50446C0
:100AA00041F65C5200212046FFF73EFB002006E0A5
:100AB00000EB40021119FF224A708A70401C40F678
:100AC000C4118842F4DB254600206870A87003201A
:100AD0002870E51C00206870A87002202870012191
:100AE00041F6585001550021401C0155401C01554C
:100AF000401C01550121C01F01512046FFF700FF96
:100B000070BD10B504462046FFF72AFF08B9002043
:100B100010BD0120FCE702460AB9002070470129F8
:100B200006DB042904DC41F6545081500120F5E72E
:100B30000020F3E7000000000000000000000000BB
:040B400000000000B1
:04000005000007658B
:00000001FF
